:020000040000FA
:020000000628D0
:0200080061296C
:04000C0004309F001D
:1000100083169F0183120C309700831603133F3021
:100020009200831204309200831647308600FF301E
:100030008500831200308500860083168101000050
:1000400081128111F830810583128B010000A60115
:10005000A60AA7019630A100C830A3000130A40071
:10006000A500AF00A201B00135282010CD20AB0AB9
:100070000319AC0A031933140314061F0310AA0D45
:100080002A080F3C031998200230A006A018A403E8
:100090000319B92001302402031D3528861856287B
:1000A000061200008612861C5328A60A2708031988
:1000B000FF28FF3E03190B29FF3E03191929FF3EB4
:1000C0000319232926080319D928FF3E03192B29D0
:1000D000FF3E03193C29FF3E03194B29FF3E03193C
:1000E0005129A6013528B00B0800FA30B0000930BC
:1000F0002E0203197E28031885288828C4302D0273
:1001000003190800031885288828A10AA2200800DE
:1001100005302E0203198F28031808009528DC30BB
:100120002D020319080003180800A103A2200800EB
:10013000B9202508A4002B08AD002C08AE00AC01A6
:10014000AB0108002108A8000330A805A80E170875
:10015000CF39280497002108FC39A8000310A80C07
:10016000280C9500080003011708CF399700950166
:10017000080006123230A8008616000000000000B9
:100180000000000000000000000000000000A80BBC
:10019000BD2886122308A40008000530A800210805
:1001A000A20703180616031C0612A80BCF28080086
:1001B0003528861CD9288612B3208618DD28A2206F
:1001C0008612A60A861CE2283528061DAF0A061CE0
:1001D000AF032F08A50725082302031C352801308B
:1001E000A50035282108FF3C0319FB28061FA10A9A
:1001F000A1080319FD28061BA103A2203528A2206F
:10020000B00B62280430B000A10A061F6228A70ABA
:100210000C30A1076228A220B00B62280A30B0007F
:10022000A103061B6228A70AFE30A1071430B20002
:100230006228A220B00B62280A30B000B20B6228FC
:10024000A70A3310622862287320A220331C622878
:10025000A101A7016228B10B35280A30B10021089D
:10026000FF3C03193529061DA10AA10803193A29E3
:10027000061CA103A2203528061DA50A2508230275
:10028000031CA501061CA503F0302502031C35281C
:100290002308A5003528A50A25082302031CA5016B
:1002A0003528A503F0302502031C35282308A500B6
:1002B0003528A50A25082302031C35280130A5008E
:0402C00035280900D4
:02400E00103F61
:00000001FF
